:1000000019C033C032C031C030C02FC02EC02DC087
:100010002CC02BC02AC029C028C027C026C025C09C
:1000200024C023C0A3C221C020C0E3C21EC01DC083
:100030001CC01BC011241FBECFEFD2E0DEBFCDBF5E
:1000400011E0A0E0B1E0E4E0FCE002C005900D9218
:10005000A433B107D9F712E0A4E3B1E001C01D92C7
:10006000A936B107E1F702D0CBC5CACF2F923F9294
:100070004F925F926F927F928F929F92BF92CF9298
:10008000DF92EF92FF920F931F93CF93DF938CEF4A
:1000900087B98FEF88B982E084B98AB98BB915B86E
:1000A00048D2A6D1789444988DE32FD186E02DD103
:1000B000449A44988CE329D183E027D1449A449808
:1000C00084E223D183E021D1449A449882E31DD174
:1000D00089E11BD1449A449881E317D189E115D174
:1000E000449A449883E211D181E00FD1449A449814
:1000F00081EE0BD1449A449880E207D18AE005D181
:10010000449A0000000000000000459A00E059E514
:10011000C52E51E0D52E40E1E42EF12C30E0232E07
:1001200031E0332E24E0822E21E0922E98E9492EF0
:100130009AE3592E8AE0682E81E0782E449887E26F
:10014000E4D08EE7E2D0449A0000000000000000F6
:1001500000000000449880EAD8D010E0812F800F82
:10016000ECD01F5F1E31D1F7449A083C11F400E037
:1001700006C0013021F480E49CE90197F1F78EEB91
:100180009AE00197F1F7449887E1BFD080E0BDD0B5
:10019000449A80FF02C00F5FD1CF449880E6B5D06B
:1001A00080E0B3D0B82E449A00000000449881E665
:1001B000ACD080E0AAD0182F813039F5809137017A
:1001C0002DB73EB7285030400FB6F8943EBF0FBE53
:1001D0002DBFEDB7FEB73196ADB7BEB71296DC9224
:1001E000CE921197F382E28235822482868317822F
:1001F00034D22DB73EB7285F3F4F0FB6F8943EBFBD
:100200000FBE2DBFA2D1109237018DB79EB70897B0
:100210000FB6F8949EBF0FBE8DBFEDB7FEB73196F7
:10022000ADB7BEB71296DC92CE921197F382E282FE
:10023000958284821683178210D22DB73EB7285F2D
:100240003F4F0FB6F8943EBF0FBE2DBF7ED110E0DA
:10025000CB2DD0E0219726C080E057D0F201319716
:10026000F1F7ADB7BEB718970FB6F894BEBF0FBE83
:10027000ADBFEDB7FEB731961296DC92CE921197D4
:10028000F382E2829582848286831782E6D12DB73B
:100290003EB7285F3F4F0FB6F8943EBF0FBE2DBF4D
:1002A00054D11F5F812F90E08C179D07ACF200D0D6
:1002B00000D000D0EDB7FEB73196ADB7BEB71296FD
:1002C000DC92CE921197F382E28275826482C5D16C
:1002D0002DB73EB72A5F3F4F0FB6F8943EBF0FBE13
:1002E0002DBF33D1449A00000000449887E20DD01E
:1002F0008EE70BD0449A00000000000000008091BF
:1003000037018F5F809337013ECF582F439890E895
:1003100040E020E030E0892F852311F0429A01C0AF
:100320004298439A3199492B439896952F5F3F4FB6
:100330002830310581F7842F0895439887FF02C044
:10034000429A01C04298439A439886FF02C0429A5B
:1003500001C04298439A439885FF02C0429A01C067
:100360004298439A439884FF02C0429A01C042983F
:10037000439A439883FF02C0429A01C04298439A2D
:10038000439882FF02C0429A01C04298439A439820
:1003900081FF02C0429A01C04298439A439880FF6D
:1003A00002C0429A01C04298439A439808954398E4
:1003B00090E880E020E030E0439A3199892B43981F
:1003C00096952F5F3F4F28303105B1F708951F9361
:1003D000162F44988062B1DF812FAFDF449A1F91BE
:1003E00008954498AADF80E090E0E1DF449A089500
:1003F000BF92CF92DF92EF92FF920F931F93449898
:1004000081E083DFB82ED3DF29E5E22E21E0F22E52
:100410002DB73EB72A5030400FB6F8943EBF0FBEFE
:100420002DBFEDB7FEB73196ADB7BEB71296FC92B1
:10043000EE92119700E110E0138302839CE0C92E35
:1004400091E0D92ED582C482B68217828087118628
:1004500004D12DB73EB7265F3F4F0FB6F8943EBF8D
:100460000FBE2DBF72D0449A449882E04EDFB82E62
:100470009EDFADB7BEB71A970FB6F894BEBF0FBEDA
:10048000ADBFEDB7FEB731961296FC92EE92119782
:1004900013830283D582C482B68217828087118635
:1004A000DCD02DB73EB7265F3F4F0FB6F8943EBF66
:1004B0000FBE2DBF4AD0449A449880E026DFB82E64
:1004C00081E023DFC82E82E020DFD82E82E01DDF0E
:1004D000ADB7BEB71E970FB6F894BEBF0FBEADBF87
:1004E000EDB7FEB731961296FC92EE9211971383F8
:1004F00002832BE131E035832483B6821782C086E4
:100500001186D286138684871586A7D02DB73EB76D
:10051000225F3F4F0FB6F8943EBF0FBE2DBF15D0E0
:10052000449A1F910F91FF90EF90DF90CF90BF9072
:1005300008951092C50089E08093C40088E98093F3
:10054000C10086E08093C200089590E007C08091CA
:10055000C00085FFFCCF9F5FE093C600E92FF0E06D
:10056000E75AFE4FE081EE2391F708951F920F9214
:100570000FB60F9211248F939F93EF93FF93909157
:10058000C600E0913401EF5FE03208F0E0E08091D6
:100590003501E81731F0E0933401F0E0E75CFE4FFD
:1005A0009083FF91EF919F918F910F900FBE0F90CD
:1005B0001F901895982F8091C00085FFFCCF9093D5
:1005C000C60008959091350180913401891711F486
:1005D00080E00895892F8F5F80933501803210F07D
:1005E00010923501E0913501F0E0E75CFE4F80812B
:1005F00008951F920F920FB60F9211248F939F931D
:10060000EF93FF93E0913601F0E0809178009091B4
:100610007900EE0FFF1FE759FE4F91838083809191
:1006200036018F5F8F7780933601FF91EF919F9115
:100630008F910F900FBE0F901F90189587E88093B1
:100640007C0010927B008DEE80937A000895F894E0
:1006500080913601789490E00895AEE0B0E0E2E356
:10066000F3E0A5C20D891E898F89988D97FF02C07E
:1006700080E090E801979E838D831A83098386E04A
:100680008C839E01255E3F4FCE010196698D7A8D48
:10069000A90111D04D815E8157FD0AC02F81388597
:1006A000421753070CF49A01020F131FF80110822E
:1006B0002E96E4E098C2ABE0B0E0E0E6F3E069C279
:1006C0003C012B015A01FC0117821682838181FDB6
:1006D00003C06FEF7FEFB9C19AE0892E1E01089425
:1006E000211C311CF3012381F20123FD859123FF9D
:1006F00081912F01882309F4A5C1853239F423FDA6
:10070000859123FF81912F01853221F490E0B3017F
:10071000B6D1E8CF982FFF24EE249924FFE1FF15EE
:10072000D0F09B3269F09C3228F4903259F0933229
:1007300091F40EC09D3249F0903369F441E024C039
:1007400052E0F52A84E0F82A28C098E0F92A25C06A
:10075000E0E1FE2A22C0F7FC29C0892F80538A30AD
:1007600070F4F6FE05C0989C902C1124980E15C0CC
:10077000E89CE02C1124E80EF0E2FF2A0EC09E3225
:1007800029F4F6FC5FC140E4F42A07C09C3619F452
:1007900050E8F52A02C0983649F4F20123FD9591FC
:1007A00023FF91912F01992309F0B8CF892F855408
:1007B000833018F08052833038F444E050E0A40EC7
:1007C000B51E5FE359830FC0933631F0933779F04C
:1007D000933509F052C01FC0F5018081898342E042
:1007E00050E0A40EB51E610101E010E011C0F5015A
:1007F000C080D180F6FC03C06FEF7FEF02C0692D8F
:1008000070E042E050E0A40EB51EC6012DD18C016F
:100810005FE7F52213C0F501C080D180F6FC03C06C
:100820006FEF7FEF02C0692D70E042E050E0A40E50
:10083000B51EC6010ED18C0150E8F52AF3FE06C0A4
:1008400018C080E290E0B3011AD1EA948E2D90E0B6
:1008500008171907B0F30DC0F601F7FC8591F7FEF4
:1008600081916F0190E0B3010AD1E110EA94015047
:1008700010400115110581F7E2C0943611F0993648
:1008800061F5F7FE08C0F501208131814281538175
:1008900084E090E00AC0F501808191819C014427A9
:1008A00037FD4095542F82E090E0A80EB91E9FE6D8
:1008B000F92257FF09C050954095309521953F4F3B
:1008C0004F4F5F4FE0E8FE2ACA01B901A1012AE0BB
:1008D00030E001D1D82ED2183FC0953729F41F2D12
:1008E0001F7E2AE030E01DC01F2D197F9F3661F06A
:1008F000903720F4983509F0A5C00FC0903739F033
:10090000983709F09FC004C028E030E00AC01061A9
:1009100014FD146020E130E004C014FD166020E1F5
:1009200032E017FF08C0F5016081718182819381F7
:1009300044E050E008C0F50180819181BC0180E075
:1009400090E042E050E0A40EB51EA101C4D0D82E24
:10095000D2188FE7F82EF122F6FE0BC05EEFF522DB
:10096000D91438F4F4FE07C0F2FC05C08FEEF8226B
:1009700002C01D2D01C0192DF4FE0DC0FE01ED0DAC
:10098000F11D8081803319F499EEF92208C01F5FB0
:10099000F2FE05C003C08F2D867809F01F5F0F2D72
:1009A000F3FC13C0F0FE0EC01E1510F09D2C0AC003
:1009B0009D2C9E0C911A1E2D05C080E290E0B30183
:1009C0005ED01F5F1E15C8F304C01E1510F4E11A97
:1009D00001C0EE2404FF0EC080E390E0B3014FD0CD
:1009E00002FF1BC001FD03C088E790E00EC088E550
:1009F00090E00BC0802F867881F001FF02C08BE26F
:100A000001C080E2F7FC8DE290E0B30138D005C070
:100A100080E390E0B30133D09A94D914C8F3DA9408
:100A2000F101ED0DF11D808190E0B30128D0DD20B2
:100A3000B1F705C080E290E0B30121D0EA94EE2046
:100A4000C9F750CEF30166817781CB012B96E2E1A5
:100A5000BCC0FC010590615070400110D8F7809532
:100A600090958E0F9F1F0895FC016150704001907A
:100A70000110D8F7809590958E0F9F1F08950F93C2
:100A80001F93CF93DF938C01EB018B8181FF1BC000
:100A900082FF0DC02E813F818C819D8128173907EF
:100AA00064F4E881F9810193F983E88306C0E8855D
:100AB000F985802F0995892B31F48E819F810196CC
:100AC0009F838E8302C00FEF1FEFC801DF91CF918C
:100AD0001F910F910895FA01AA27283051F1203172
:100AE00081F1E8946F936E7F6E5F7F4F8F4F9F4FC2
:100AF000AF4FB1E03ED0B4E03CD0670F781F891F04
:100B00009A1FA11D680F791F8A1F911DA11D6A0FD1
:100B1000711D811D911DA11D20D009F468943F9184
:100B20002AE0269F11243019305D3193DEF6CF0183
:100B30000895462F4770405D4193B3E00FD0C9F749
:100B4000F6CF462F4F70405D4A3318F0495D31FDB6
:100B50004052419302D0A9F7EACFB4E0A695979509
:100B6000879577956795BA95C9F7009761057105DF
:100B700008959B01AC010A2E069457954795379529
:100B80002795BA95C9F7620F731F841F951FA01D83
:100B900008952F923F924F925F926F927F928F9221
:100BA0009F92AF92BF92CF92DF92EF92FF920F93FC
:100BB0001F93CF93DF93CDB7DEB7CA1BDB0B0FB606
:100BC000F894DEBF0FBECDBF09942A8839884888C3
:100BD0005F846E847D848C849B84AA84B984C88459
:100BE000DF80EE80FD800C811B81AA81B981CE0F50
:100BF000D11D0FB6F894DEBF0FBECDBFED01089535
:040C0000F894FFCF96
:100C040025640A002530327820000A0053543A2023
:100C14002530325820253032580A0053543A2025C2
:100C24003032582025303258202530325820253093
:040C340032780A0008
:00000001FF
